:020000040800F2
:1000000058050020D90000083112000861110008CD
:1000100000000000000000000000000000000000E0
:100020000000000000000000000000007B1200083B
:100030000000000000000000791200087D12000896
:10004000EB000008EB000008EB000008EB000008E4
:10005000EB000008EB000008EB000008EB000008D4
:1000600000000000EB000008EB000008EB000008B7
:10007000EB000008EB00000800000000EB000008A7
:1000800000000000EB00000800000000000000007D
:10009000EB00000800000000EB000008EB00000887
:1000A000EB000008EB000008EB0000083D1800081A
:1000B0004D180008EB0000080000000000000000E0
:1000C0000448854600F090F800480047A51900084C
:1000D000C046C046580500200448804704480047F1
:1000E000FEE7FEE7FEE7FEE7FEE7FEE7F5120008A3
:1000F000C100000830B50B46014600202022012433
:1001000009E00D46D5409D4205D31D469540491B4B
:100110002546954040191546521E002DF1DC30BD94
:10012000F0B51FB40646002082B005464024019178
:1001300000901BE0019922460F46304600F042F83D
:10014000049A059B801A994110D3104619462246FD
:1001500000F028F8361A8F4101972246012000212D
:10016000009F00F01FF838184D4100902046641E93
:100170000028DFDC019B00982946324607B0F0BD1D
:10018000D2B201E00270401C491EFBD2704700222F
:10019000F6E710B513460A4604461946FFF7F0FF86
:1001A000204610BD10B5202A04DB0146203A9140BC
:1001B000002010BD914020239C1A0346E3401943C0
:1001C000904010BD10B5202A04DB0846203AD040EC
:1001D000002110BD0B46D340D0402024A21A9140EC
:1001E0000843194610BD0000064C0125064E05E0E7
:1001F000E36807CC2B430C3C98471034B442F7D348
:10020000FFF762FF0C1A00082C1A0008704770B53F
:100210000024014620314A79022A03D00421C16317
:10022000012418E0026813680E25AB4313600268CE
:1002300013685B085B001360436C1C2213400122AF
:1002400015469D40036C5D604A7100220A71816B06
:10025000002900D08847204670BD0000F8B5002373
:100260000124A2E027469F403A4070D04D68022DFD
:1002700001D0122D14D1DD08AD002D1800952D6A86
:100280005E07AC46F50E0F26AE46AE406546B5435A
:10029000AC460E697546AE4065462E43009D2E6203
:1002A0004D68012D05D0022D03D0112D01D0122D46
:1002B00016D185680326AC465D00AE46AE40654665
:1002C000B543AC46CE687546AE4065462E43866063
:1002D00046680D79BE43ED06ED0F9D403543456000
:1002E00006685F000325BD40AE46AE430D79B446B7
:1002F000AE07B60FBE4065462E430660C66875461B
:10030000AE438D68BD403543C5604D68ED004BD5AB
:10031000294D6E6B26436E639E08284DB6007519F5
:10032000AC46AD689E07360F0F27B740BD43052783
:100330003F07B84201D1002715E0214FB84201D153
:10034000012710E01F4FB84202D102270BE02BE03B
:100350001D4FB84201D1032705E01C4FB84201D11F
:10036000052700E00627B7402F436546AF60184DCC
:100370002E684F689643FF0300D516432E606E68C3
:100380004F689643BF0300D516436E60AE684F6852
:100390009643FF0200D51643AE60EE684F68964361
:1003A000BF0200D51643EE605B1C0A681546DD40AF
:1003B00000D057E7F8BD00000010024000000140E7
:1003C0000004005000080050000C0050001C0050B9
:1003D0000004014001480068704700001000002040
:1003E00002480168491C01607047000010000020AD
:1003F00010B50848002401684022114301602046DE
:1004000000F00AF8002801D0012401E000F01CF8F7
:10041000204610BD0020024070B5054609487D21E8
:100420000024C9000068FFF765FE00F0F9FB002812
:1004300001D0012404E000222946501E00F01AF8E1
:10044000204670BD140000200448416B0122114376
:100450004163816B020411438163704700100240C5
:10046000C106C90E0120884001490860704700009C
:1004700000E100E010B500F0DDFE10BDF8B5044667
:100480000078544D800672D5524E0027403EB06B26
:10049000C00004D4B06BA9050843B06301274E48DF
:1004A0000168C90511D40168821511430160FFF785
:1004B00091FF009005E0FFF78DFF0099401A642836
:1004C00037D845480068C005F5D5326803210905CD
:1004D00060680A400140914208D08103890F0329D6
:1004E00004D13168890301D50120F8BD2A690321AF
:1004F00009040A4022D0084090421FD0207880068C
:100500001CD528692A6988430121C9040A432A6144
:100510002A698A432A612861C0050FD5FFF75AFF6F
:10052000009008E0FFF756FF0099411A2B488142DE
:1005300001D90320F8BD28698005F3D561688803D7
:10054000800F032805D132680005824301400A4329
:10055000326028690322616812041140084328614F
:10056000002F04D0B16B012000078143B1632078D4
:10057000C00705D0E868A168800880000843E860EB
:100580002078800705D5E8680C218843E168084396
:10059000E8602078400706D5E8680321890288438F
:1005A00021690843E8602078000706D5E868032140
:1005B0000903884361690843E8602078000606D58E
:1005C000E868032189048843A1690843E8600020A2
:1005D000F8BD000040100240007000408813000089
:1005E000F8B50E4605007DD053480068C007C00F1F
:1005F000B0420AD2504801684908490031430160BD
:100600000068C007C00FB04271D128784B4C8007FA
:1006100005D5E068F0218843A9680843E0602878A0
:10062000C00752D06868022817D0032818D0216864
:10063000012818D08905002959DAE168890889005C
:100640000143E160FFF7C6FE69680746022912D040
:1006500003291CD0012926D033E021688903EAE769
:1006600021688901E7E74907E5E7FFF7B3FEC11B0A
:100670003348814223D8E0680007800F0228F4D174
:1006800023E0FFF7A7FEC11B2D48814217D8E06881
:100690000007800F0328F4D117E0FFF79BFEC11B72
:1006A000274881420BD8E0680007800F0128F4D169
:1006B0000BE0FFF78FFEC11B2148814201D90320C7
:1006C000F8BDE0680007800FF3D11B480168C90737
:1006D000C90FB1420DD90168490849003143016091
:1006E000006800E003E0C007C00FB04201D0012065
:1006F000F8BD2878400706D5E0680721090288433D
:10070000E9680843E0602878000707D5E06807211A
:10071000C90288432969C9000843E06000F036F83F
:10072000E168084A0906090F515CC840064908609B
:100730000020FFF771FEF8BD0020024000100240CB
:1007400088130000E8190008140000200448054937
:100750000068C968044A4905490F515CC8407047A0
:100760001400002000100240011A00080448054946
:100770000068C968044A8904490F515CC840704741
:100780001400002000100240011A000810B5184A99
:10079000D1680C20084004280BD0082810D00C2861
:1007A00010D050680004410F0120C003491C88404C
:1007B00010BD1068C00601D50E4810BD0E4810BD12
:1007C0000E4810BD88020E4B000F185C0902D3685A
:1007D000890F491CDB0301D5084A05E01268D206DF
:1007E00001D5044A00E0044A5043FFF783FC10BDE2
:1007F0000010024000093D000024F40000127A00BD
:10080000F8190008FEB505007ED0FE4CE7680C2004
:10081000E66807400120000406402878C00747D05A
:10082000082F05D00C2F0AD101200004864206D1E2
:10083000206880033CD568680028E5D038E00120B6
:1008400069680004814203D121680143216011E0FD
:10085000052301221B0492049942216802D111430D
:100860002160F1E781432160216801400091206807
:1008700090432060686800280DD0FFF7ABFD009022
:1008800005E0FFF7A7FD0099401A64287AD8206890
:100890008003F6D50CE0FFF79DFD009005E0FFF723
:1008A00099FD0099401A6428F0D820688003F6D496
:1008B0002878800755D50923E868042F0DD00C2F20
:1008C00001D1002E09D000283BD021689943014373
:1008D0002160FFF77FFD064627E02168490701D523
:1008E000002891D061681F22120291432A691202E6
:1008F000114361602168994301432160FFF746FF7E
:10090000E16809060A0F00E079E1BF49895CC84047
:10091000BE4908600020FFF77FFD002872D120E06B
:10092000FFF758FD801B0228B0D820684007F7D594
:1009300060681F2109028843296909020843606031
:100940000FE02068400840002060FFF743FD0646A6
:1009500004E0FFF73FFD801B022897D8206840077E
:10096000F7D42878C0065FD5002F0CD0A8690028DE
:1009700049D02068FF21013108432060FFF72AFD9C
:1009800006462DE0C0E02068800502D5A869002851
:10099000A7D06068072149038843296A084360603B
:1009A0006068297F0002000A090608436060286A1F
:1009B000410B0120C003491C8840E16809060A0F69
:1009C0009149895CC840914908600020FFF724FDE7
:1009D000002817D128E0FFF7FDFC801B0228A3D8D0
:1009E00020688005F7D56068072149038843296A94
:1009F000084360606068297F0002000A0906084316
:100A0000606011E0E1E02168FF2001308143216056
:100A1000FFF7E0FC064604E0FFF7DCFC801B022841
:100A200072D820688005F7D42878794E000724D53D
:100A300068690028306910D0012108433061FFF750
:100A4000C9FC009005E0FFF7C5FC0099401A022898
:100A50005AD830698007F6D50FE040084000306171
:100A6000FFF7B8FC009005E0FFF7B4FC0099401ACE
:100A7000022849D830698007F6D42878400765D520
:100A800000200290A06BC00006D4A06B01210907D2
:100A90000843A063012002905E480168C90511D493
:100AA0000168821511430160FFF794FC009005E096
:100AB000FFF790FC0099401A642825D85548006833
:100AC000C005F5D5FF20AA680130824203D1316903
:100AD0000143316111E001218902002A07D0052379
:100AE0001B029A4203D132690A433261EFE732694D
:100AF00082433261306988433061A86800280FD092
:100B0000FFF768FC009007E05EE0FFF763FC0099E8
:100B1000411A4148814257D830698005F5D50DE02A
:100B2000FFF758FC009006E0FFF754FC0099411ACB
:100B30003948814248D830698005F5D402980028A8
:100B400004D0A06B012109078843A063686A0028CC
:100B500064D00C2F3ED0012636060228206805D02E
:100B6000B0432060FFF736FC05462FE0B04320601D
:100B7000FFF730FC074604E0FFF72CFCC01B0228FF
:100B800022D820688001F7D4E96AA86AE26808439D
:100B9000296BFD231B049A4311430843E06020683E
:100BA00030432060FFF716FC054604E0FFF712FC17
:100BB000401B022808D820688001F7D52EE0FFF7F7
:100BC00009FC401B022801D90320FEBD20688001DA
:100BD000F5D423E00128F8D0E06801210904AA6ACD
:100BE000014091420BD10F218904EA6A01409142F0
:100BF00005D1032189050840296B88420ED00120C8
:100C0000FEBD000000100240E8190008140000209A
:100C10004010024000700040881300000020EFE701
:100C2000094910B5401E884201D9012010BD074C6A
:100C300060610321081F00F0FDFA0020A061072079
:100C40002061002010BD0000FFFFFF0000E000E079
:100C5000F0B502462032137E012B15D001271776FE
:100C60000223537605686C68AB687026B4430E683F
:100C7000496826438024A34319436E60006881605D
:100C8000577600201076F0BD0220F0BD70B504004C
:100C900005D025462035687E002802D006E00120D8
:100CA00070BD00202876204600F00AF80220687601
:100CB000211D206800F048FB01206876002070BDEF
:100CC00000680449884204D10348816B1022114313
:100CD0008163704700100040001002407047704769
:100CE000F8B502680446D0691168936805072D0FAE
:100CF0005BD0DD07ED0FFF2621360E402E4367D077
:100D0000C60706D0CE0504D501261662E26F32432F
:100D1000E267870702220426002F06DADF0704D0E5
:100D200027683A62E76F3743E767470706D5DB076F
:100D300004D023681E62E36F1343E367020709D5FB
:100D400020220A402A4305D0236808221A62E36F52
:100D50001343E367E26F002A2FD0800606D588068A
:100D600004D5216E002901D020468847E06F216814
:100D70008968490601D4000724D5204600F0B0FB5D
:100D800020688168490619D58168402291438160B5
:100D9000E06E002812D020498163E06EFFF737FA39
:100DA00000280AD0E06E816B06E0850610D58D061E
:100DB0000ED5216E1CE020468847F8BD2046FFF77F
:100DC0008EFFF8BD2046FFF78AFF0020E067F8BDE0
:100DD000C50208D55B0206D5012000051062204639
:100DE000FFF77CFFF8BD030605D50B0603D5616E42
:100DF0000029E0D1F8BD4006FCD54806FAD51368B5
:100E0000204640218B4313602021616700216166E9
:100E100000F0A5F9F8BD0000CD14000810B50400DD
:100E200003D0606F002802D007E0012010BD002130
:100E300070200155204600F027F8242060672068C4
:100E40000168490849000160204600F0B1FB012813
:100E5000ECD0606A002802D0204600F0A1FA206899
:100E600041680922D20291434160206881682A22A8
:100E7000914381602068016801221143016020468E
:100E800000F0F4FA10BD0000F0B587B0044614215C
:100E90006846FFF77CF9244F266800212348012289
:100EA000022303240425BE421AD1466B97033E4316
:100EB0004663C66A1643C662C06A02AE1040059019
:100EC00060020090019332C6052069460007FFF7D3
:100ED000C5F9002211461B20FFF7CCFA1B201EE0AB
:100EE000134FBE421DD1866B01277F043E438663AC
:100EF000C66A1643C662C06A02AEC007C00F05903C
:100F00000C200090019332C6052069460007FFF7C8
:100F1000A5F9002211461C20FFF7ACFA1C20FFF7B0
:100F20009FFA07B0F0BD00000038014000100240F9
:100F300000440040F0B5836F202B54D100290AD023
:100F4000002A08D08568DC01A54206D10369002B80
:100F500003D1CB0701D00120F0BD034660331E7CD6
:100F6000012E40D001261E744165014640310A839E
:100F70004A830022FF260266A54204D10569002D9E
:100F800013D11A4D0AE07F27002D09D0012636071C
:100F9000B5420CD10569002D05D03F258D8307E0B2
:100FA0000569002D01D08F8302E08E8300E08A83E3
:100FB000C2672221816701688D68012635438D60F3
:100FC0008168A14202D1016900290AD0084901665D
:100FD0001A7400680168FF22213211430160002069
:100FE000F0BD0449F3E70220F0BD0000FF0100005E
:100FF000591500080115000810B5006820498842FD
:1010000024D1204C21780D2921D01FA000F026FCEE
:1010100061780D291FD01CA000F020FCA1780D29BB
:101020001DD019A000F01AFCE1780D291BD016A0E4
:1010300000F014FC21790D2919D013A000F00EFC4A
:1010400061790D2917D010A000F008FC10BD0FA089
:1010500000F004FCDCE70DA000F000FCDEE70BA0D4
:1010600000F0FCFBE0E709A000F0F8FBE2E707A0D6
:1010700000F0F4FBE4E705A000F0F0FB10BD000079
:101080000044004000000020256300000A0000002A
:10109000FFB50446406F83B017460D4620285CD14B
:1010A000002D0AD0002F08D0A168C001814207D1CD
:1010B0002069002804D1E80702D0012007B0F0BD64
:1010C000204660300290007C012846D00298012121
:1010D00001740020E06721206067FFF77BF9264656
:1010E00040360190378277820120A1680003814257
:1010F00002D12069002802D02F46002511E00027E8
:101100000FE000228021204600F066FB002815D168
:10111000002F15D02168387888627F1C708A401EA5
:101120007082708A019B002806980090E9D1002205
:101130004021204600F050FB002808D00320BDE7E6
:1011400028882168C005C00D8862AD1CE6E7202014
:101150006067029900200874B0E70220AEE770478C
:10116000FEE7000008B50448C16A01221143C162CC
:10117000C06A1040009008BD001002401CB5002459
:101180000E4800940C49019401600721846041607D
:1011900001214461C160FFF779FD002801D0FFF70C
:1011A00035F80094694605480194FFF751FD002881
:1011B00001D0FFF72BF81CBD001000401C000020E0
:1011C00010B50C480A490160E12149024160002143
:1011D0008160C16001618161C1610C220162426173
:1011E0004162FFF71BFE002801D0FFF70FF810BD8A
:1011F000003801405800002010B50C480A49016031
:101200004B21C901416000218160C16001618161A0
:10121000C1610C22016242614162FFF7FFFD0028BB
:1012200001D0FEF7F3FF10BD00440040D8000020BD
:10123000704700008307FF22DB0E9A408907090EE2
:10124000994000280BDA0007000F08388308084887
:101250009B001818C36993430B43C361704783080D
:1012600004489B001B181868904308431860704797
:1012700000ED00E000E400E07047704710B5FFF7B4
:10128000AFF810BD30B599B034216846FEF77FFF46
:1012900014210DA8FEF77BFF1C2112A8FEF777FF93
:1012A000134801680322D2029143C21489180160D5
:1012B0000220009000241020099401250490039539
:1012C0006846FFF79FFA0F200D9080200F900E9533
:1012D0001094002111940DA8FFF782F903201290B9
:1012E0001494159412A8FFF7C9F819B030BD000086
:1012F0000070004010480168821511430160C16808
:101300000E4A1140C16001680D4A114001608168B8
:1013100049084900816001680122920491430160FB
:10132000C168FD2212049143C16000210161054999
:10133000C003886070470000001002400C40FF8826
:10134000F6FFF6FE00ED00E070B5026801239B0792
:10135000114C124D984203D0A04201D0A84203D1B3
:101360007026B2434E683243984203D0A04201D067
:10137000A84204D103231B029A43CB681A4380235B
:101380009A430B691A4302608A68C26209688162E3
:101390000121416170BD00000008014000140140BE
:1013A00010B5818CC90707D001684A6801235B0426
:1013B0009A43836A1A434A60818C890707D501687A
:1013C0004A6801231B049A43C36A1A434A60818C0A
:1013D000490707D501684A6801239B049A43036BB8
:1013E0001A434A60818C090707D501684A680123BE
:1013F000DB039A43436B1A434A60818CC90607D5C5
:101400000268916801231B039943836B1943916020
:10141000818C890607D501688A6801235B039A439A
:10142000C36B1A438A60818C490612D503685A68D7
:1014300001210905046C8A4322435A60026C8A42E6
:1014400007D10268516803235B059943436C194334
:101450005160818C090607D501684A680123DB04C5
:10146000806C9A4302434A6010BD0000F8B5002624
:101470000446C667FEF7AEFF054620680068124FB7
:10148000000709D501212B46002249052046009777
:1014900000F0A2F900280DD12068006840070BD5A4
:1014A00001212B46002289052046009700F094F97F
:1014B000002801D00320F8BD20206067A0676034B9
:1014C00026740020F8BD0000FFFFFF0110B5806A00
:1014D0000022014640314A834A82FFF700FC10BDDA
:1014E00001680A68FF2321339A430A6001688A6809
:1014F000520852008A6020218167002101667047EE
:1015000010B5014640318B8B846F0268222C04D0C9
:10151000906908210843906110BD526A446D1A40D9
:101520002280426D921C42654A8B521E4A83498B2F
:101530000029F1D101680A68FF2321339A430A6028
:1015400001688A68520852008A6020218167002160
:101550000166FFF751FD10BD10B5014640318B8B80
:10156000846F0268222C04D090690821084390619E
:1015700010BD526A1A40436D1A70426D521C42658A
:101580004A8B521E4A83498B0029F1D101680A68AF
:10159000FF2321339A430A6001688A685208520087
:1015A0008A602021816700210166FFF725FD10BDBB
:1015B000F8B504462669A268E769324366691020D7
:1015C00000253E432368324378491E68784F3E40E9
:1015D00016431E6023685A6803263603B243E66842
:1015E00032435A602368A2698B4201D0266A324393
:1015F0009E680B273F02BE4316439E606D4E2368D4
:101600006D4AB3420CD1D2689207920F06D0012ADC
:1016100038D0022A34D0032A20D11EE001201DE058
:10162000664EB3420AD1D2680C26324026D0042A34
:1016300028D0082A24D00C2A10D10EE08B420DD1DC
:10164000D66803229202164018D001229202B61ADE
:1016500018D0B61A14D0964200D10820564A012656
:10166000403A574FF6038B4236D100280CD002285F
:101670000DD0042812D008281FD11CE00020EDE76F
:101680000220EBE70420E9E7FFF760F808E01068C4
:10169000C00601D5384605E04A4803E0FFF776F872
:1016A000002873D0626851005118814205D8110397
:1016B000814202D303E03046F4E7012566E0010EE3
:1016C00006025008002330185941FEF729FD032176
:1016D0000902411A3C4A55E0E169B14232D10300A6
:1016E00000F0CCF809070A0D06250606062B0600B1
:1016F000E3E7FFF72BF81CE0FFF738F819E0106874
:101700006168C00602D54808304A01E0304A4808FE
:101710008018FEF7EFFC80B201462E4A1039914244
:10172000CBD8511C01400007400F08432CE0FFF7C5
:101730002DF8616840004A08EAE76168012248081C
:101740001204E5E7030000F099F809070A0D0626E0
:101750000606062C0600B0E7FEF7F8FF1DE0FFF7CF
:1017600005F81AE010686168C00602D54808C0197B
:1017700002E014484A081018FEF7BCFC80B201468B
:10178000144A1039914298D82168C8600020206618
:1017900060662846F8BDFEF7F9FF61684A088018C0
:1017A000EAE7616848088019E6E700000048004061
:1017B000F369FFEF00380140401002400044004050
:1017C00000093D000024F400FFFC0F0000127A0025
:1017D0000048E801EFFF0000FFB581B017460E4654
:1017E00004460A9D09E0681C07D0FEF7F3FD049942
:1017F000401AA8420CD8002D0AD02068C169304692
:10180000884318D00020B842EDD0002005B0F0BDCC
:1018100020680168FF22A13291430160206881683D
:1018200049084900816020206067A067002060347B
:1018300020740320EAE70120E5E7000010B5024824
:10184000FFF74EFA10BD00005800002010B5024806
:10185000FFF746FA10BD0000D80000200FB410B505
:1018600003A9044B044A029800F024F810BC08BCF9
:1018700004B01847891900081800002030B47446D5
:10188000641E2578641CAB4200D21D46635D5B007C
:10189000E31830BC184702E008C8121F08C1002A2C
:1018A000FAD170477047002001E001C1121F002AE1
:1018B000FBD17047FFB581B00546002706E025281B
:1018C0000AD0049A039990476D1C7F1C2878002841
:1018D000F5D1384605B0F0BD002269786D1C104680
:1018E0002E2913D1697804226D1C2A2909D1029965
:1018F0006D1C01C9029109E00A23584330380818C9
:101900006D1C29780B46303B092BF5D92B78002B21
:10191000DFD0632B07D0732B10D0049A184603999D
:1019200090477F1C2DE002996C460B782370091DAF
:101930000291002161706E46012104E0029940C9C4
:1019400002910021C94352070AD5002400E0641C1B
:1019500084420DDA8C42FADB325D002AF7D107E0CF
:10196000002400E0641C8C42FCDB305D0028F9D1CF
:101970003F1904E03078049A761C03999047641E5E
:10198000F8D26D1CA2E7000001B5044B01226946A4
:101990000348FFF77DFB009808BD0000FFFF000033
:1019A00058000020FEF724FDFFF76CFCFFF7DAFB80
:1019B000FFF706FCFFF7E2FBFFF71EFC064B0822D1
:1019C00006490748FFF764FB04490622891F0548BA
:1019D000FFF7B0FAF8E70000FFFF00000600002064
:1019E00058000020D8000020000000000000000087
:1019F0000102030406070809030406080C10182056
:101A00003000000000010203040000002C1A00084E
:101A1000000000201C00000096180008481A00086A
:101A20001C0000203C050000A61800080000000073
:101A3000000043616C2C647279000000000000001B
:081A400000002000000000007E
:04000005080000C12E
:00000001FF
